S31508008000E83F00209D820008A9820008AB8200088C
S31508008010AD820008AF820008B182000800000000A7
S31508008020000000000000000000000000B382000805
S31508008030B582000800000000B7820008099F000802
S31508008040BB820008BB820008BB820008BB8200080E
S31508008050BB820008BB820008BB820008BB820008FE
S31508008060BB820008BB820008BB820008BB820008EE
S31508008070BB820008BB820008BB820008BB820008DE
S31508008080BB820008BB820008BB820008BB820008CE
S31508008090BB820008BB820008BB820008BB820008BE
S315080080A0BB820008BB820008BB820008BB820008AE
S315080080B0BB820008BB820008BB820008BB8200089E
S315080080C0BB820008BB820008BB820008BB8200088E
S315080080D0BB820008BB820008BB820008BB8200087E
S315080080E0BB820008BB820008BB820008BB8200086E
S315080080F0BB820008BB820008BB820008BB8200085E
S31508008100BB820008BB820008BB820008BB8200084D
S31508008110BB820008BB820008BB820008BB8200083D
S31508008120BB820008BB820008BB820008BB8200082D
S31508008130BB820008BB820008BB820008BB8200081D
S31508008140BB820008BB820008BB820008BB8200080D
S31508008150BB820008BB820008BB820008BB820008FD
S31508008160BB820008BB820008BB820008BB820008ED
S31508008170BB820008BB820008BB8200080000000022
S31508008180BB820008BB820008BB820008BB820008CD
S31508008190BB820008BB820008BB820008BB820008BD
S315080081A0BB820008BB820008BB820008BB820008AD
S315080081B0BB820008BB820008BB820008BB8200089D
S315080081C0BB820008BB82000800000000BB820008D2
S315080081D0BB820008BB820008BB820008BB8200087D
S315080081E0BB820008BB820008BB820008BB8200086D
S315080081F0BB820008BB820008EE11AA5500F002F8FF
S3150800820000F03CF80AA090E8000C82448344AAF1E6
S315080082100107DA4501D100F031F8AFF2090EBAE8E4
S315080082200F0013F0010F18BFFB1A43F0010318479C
S31508008230D4370000F4370000103A24BF78C878C154
S31508008240FAD8520724BF30C830C144BF04680C604E
S31508008250704700000023002400250026103A28BF96
S3150800826078C1FBD8520728BF30C148BF0B6070479A
S315080082701FB503F0AFFB1FBD10B510BD00F0A0F988
S315080082801146FFF7F5FF02F0DCFA00F0BEF903B479
S31508008290FFF7F2FF03BC00F0C5F900000A4885465F
S315080082A00A4880470A480047FEE7FEE7FEE7FEE77A
S315080082B0FEE7FEE7FEE7FEE7FEE7FEE705480649B6
S315080082C0064A074B70470000E83F0020A19F0008B8
S315080082D0FD810008E8390020E83F0020E83B00203F
S315080082E0E83B002053EA020C00F069802DE9F04BC8
S315080082F04FF00006002B1FBFB3FA83F503FA05F407
S3150800830024FA05F65E4012BF1643B2FA82F502FA5F
S3150800831005F4C5F120051EBF22FA05FC44EA0C0443
S31508008320203556EA044C4FEA144418BF641C4FF033
S3150800833000084FF00009904271EB030C39D300296D
S3150800834019BFB1FA81F701FA07F6B0FA80F700FA11
S3150800835007F6C7F120071EBF20FA07FC46EA0C06F7
S315080083602037B6FBF4FCA7EB0507103F07F01F0BF9
S31508008370CBF120060CFA0BFB2CFA06F644BFB346E3
S315080083800026202FA4BF5E464FF0000B5BEA060CC2
S3150800839008BF4FF0010B19EB0B09ABFB027C48EB4E
S315080083A00608C01B06FB02CC0BFB03CC71EB0C01C9
S315080083B0C1E70B46024641464846BDE8F08B13B571
S315080083C04FF000004FF00001AFF30080BDE81C40FD
S315080083D0704740EA010310B59B070FD1042A0DD355
S315080083E010C808C9121F9C42F8D020BA19BA884288
S315080083F001D9012010BD4FF0FF3010BD1AB1D307C7
S3150800840003D0521C07E0002010BD10F8013B11F8FC
S31508008410014B1B1B07D110F8013B11F8014B1B1B25
S3150800842001D1921EF1D1184610BD032A40F23080C0
S3150800843010F0030C00F0158011F8013BBCF1020F97
S31508008440624498BF11F801CB00F8013B38BF11F818
S31508008450013BA2F1040298BF00F801CB38BF00F82F
S31508008460013B11F0030300F05280083AC0F008807F
S3150800847051F8043B083A51F804CBA0E80810F5E790
S31508008480121D5CBF51F8043B40F8043BAFF3008073
S31508008490D20724BF11F8013B11F801CB48BF11F8E8
S315080084A0012B24BF00F8013B00F801CB48BF00F8B8
S315080084B0012B704702F0FF0343EA032242EA024215
S315080084C000F002B84FF000020429C0F0128010F044
S315080084D0030C00F05080CCF1040CBCF1020F18BF5D
S315080084E000F8012BA8BF20F8022BA1EB0C0100F025
S315080084F042B85FEAC17C24BF00F8012B00F8012BC3
S3150800850048BF00F8012B704770477047704710B591
S31508008510203AC0F00B80B1E81850203AA0E818506D
S31508008520B1E81850A0E81850BFF4F5AF5FEA027C2E
S3150800853024BFB1E81850A0E8185044BF18C918C09D
S31508008540BDE810405FEA827C24BF51F8043B40F83E
S31508008550043B08BF7047D20728BF31F8023B48BF23
S3150800856011F8012B28BF20F8023B48BF00F8012B61
S3150800857070474FF0000200B51346944696462039D8
S3150800858022BFA0E80C50A0E80C50B1F12001BFF4BE
S31508008590F7AF090728BFA0E80C5048BF0CC05DF824
S315080085A004EB890028BF40F8042B08BF704748BF72
S315080085B020F8022B11F0804F18BF00F8012B7047E6
S315080085C0754600F02BF8AE4605006946534620F07E
S315080085D00700854618B020B5FFF770FEBDE82040B5
S315080085E04FF000064FF000074FF000084FF0000B61
S315080085F021F00701AC46ACE8C009ACE8C009ACE814
S31508008600C009ACE8C0098D46704710B50446AFF3FB
S3150800861000802046BDE81040FFF739BE0048704785
S315080086208839002001491820ABBEFEE72600020063
S3150800863070470000BFF34F8F05480168054A01F4EB
S31508008640E06111430160BFF34F8F00BFFDE70000F3
S315080086500CED00E00400FA0500F002B800F03AB8A4
S3150800866070B51A4C00251A4E607800280ED020786E
S315080086703044401C01F002FF012817D001F0B6FC77
S3150800868061686431884200D9657070BD104801F090
S31508008690F5FE0128F9D13078401E3F28F5D801F0BB
S315080086A0A5FC606001206070257070BD2078401CB4
S315080086B0C0B2207031788142F7D165707078FF2892
S315080086C0F3D1B0780028F0D1FFF7B4FF58000020A6
S315080086D0A03100200948084901604FF46141416012
S315080086E000218160C16001610C2242618161C16122
S315080086F00162416201F0D1B900480040E43100202E
S31508008700006800F58050816941F002018161704777
S31508008710006800F58050816941F400518161704715
S3150800872038B50446206800F58050816941F4801107
S315080087308161206800F5805080690090012000F072
S3150800874007F92068009900F58050816138BD00005E
S315080087505379107940EA0323074808440364D37819
S31508008760117841EA0361937852781B0443EA02229E
S315080087701143416470470000008002402DE9F04132
S31508008780AEB00446002904D04FF40060E060C00093
S31508008790A0600025119512951395149515951695B3
S315080087A0E06900287DD017954FF400701890199548
S315080087B01A951B951C951D9540271E971F95209564
S315080087C021952295239524952595269580262796E5
S315080087D0289529952A952B952C952D95206802681C
S315080087E045490A40D4E902131943179B194341F432
S315080087F00071114301602068D0F80080012000F064
S31508008800A7F82068C0F80080206847602068476895
S31508008810012000F09DF82068476020688560206880
S31508008820C560206881694FF64172114041F08001A8
S31508008830816120688769012000F08AF820688761CD
S315080088402068C5612068C769012000F081F82068A2
S31508008850C7610195B004029003950111049105952D
S31508008860069507950895042109910A9040120B90E0
S3150800887080010C9040120D900E960F951095206869
S3150800888000F5805081691D4A11401D4A0A438261DC
S31508008890206800F580508569012000F059F82068A5
S315080088A000E016E000F5805085612068154900F55E
S315080088B080500160206800F580500568012000F0AE
S315080088C047F8206800F580500560A069012804D0A3
S315080088D00AE04FF48060179066E7206800F580503C
S315080088E0C169094A1143C16162692EB02046002157
S315080088F0BDE8F041FFF72CBF0F8120FF233FDEF8CC
S31508008900040020028020C1024000010038B5044658
S315080089102068016841F00401016020680068009041
S31508008920012000F015F821680098086038BD38B5B0
S3150800893004462068016841F0080101602068006863
S315080089400090012000F004F821680098086038BDFE
S3150800895070B5044600F054FC0546601C02D0044875
S315080089600078044400F04CFC401BA042FAD370BDCA
S3150800897040000020F0B5002490F84550012D09D09C
S31508008980012780F84570022580F84450816244F238
S31508008990F45C19E00220F0BD01EB44154FF00046E7
S315080089A02E60C5F804C0C4EBC41606EB460602EBF7
S315080089B08606AE6086695E1EB44203D205F12006BD
S315080089C0EE6000E0E960641C9C42E5D3026802F5AB
S315080089D08052D16080F84470002180F8451000204C
S315080089E0F0BD2DE9F043002590F84540012C0BD049
S315080089F04FF0010C80F845C0022480F84440C1625B
S31508008A005F1E4FF480181CE00220BDE8F08301EBDE
S31508008A104514C4F80080C5EBC51606EB460602EBFE
S31508008A208606A660C66926B9266846F44009C4F8CB
S31508008A300090BD4203D204F12006E66000E0E16042
S31508008A406D1C9D42E3D3026802F58052116180F8DD
S31508008A5044C0002180F845100020D6E710B590F8EC
S31508008A604510012913D0012380F84530022180F8EA
S31508008A704410816A0A680024002A29DB0A68D2059C
S31508008A8018D5826B521C8263012A02D002E00220AA
S31508008A9010BD01632830C1600A68C2F30D42121F77
S31508008AA04261826892688261C96801600377447787
S31508008AB0002010BD0A68920505D5016344638363E7
S31508008AC0C968816204E0826B521C8263C96881624C
S31508008AD000F8443F4470012010BD00002DE9FC4712
S31508008AE0044600260196B046002C03D094F84400AC
S31508008AF018B107E00120BDE8FC8784F845602046E8
S31508008B0000F002F97648016841F480410160006886
S31508008B1000F4804000907348016821F40001016068
S31508008B200168226A11430160206800F580500168D7
S31508008B3041F00101016000F063FB05464FF4FA7746
S31508008B4009E000F05DFB401BB84204D9032004F895
S31508008B50440F6670CFE7206800F580500068C007AC
S31508008B60EFD12068006920F01C0500F027FD5E495A
S31508008B705E4A0144914202D245F0080516E05C4976
S31508008B805C4A0144914202D245F00C050EE05A496E
S31508008B905A4A0144914209D35949084459498842D5
S31508008BA002D245F0040501E045F01005206805618C
S31508008BB000214FF40042204600F0ECF9012538B1B7
S31508008BC001212046FFF7DAFD84F84450012092E798
S31508008BD0FF20FFF7BDFE6068F0B300F011FB074603
S31508008BE041F288390121204601AA00F0E7F800F091
S31508008BF007FBC01B484508D901212046FFF7BEFDE3
S31508008C0004F8445F6670032075E701984007E9D5C4
S31508008C10002120464FF4805200F0BCF938B10121FA
S31508008C202046FFF7ABFD84F84450012063E700F0C7
S31508008C30E7FA07462046012101AA00F0BFF800F02E
S31508008C40DFFAC01B48450AD901212046FFF796FDE1
S31508008C5004F8445F667000E022E003204BE70198C1
S31508008C608006E7D51021204601AA00F0A7F838B1FA
S31508008C7001212046FFF782FD84F8445001203AE797
S31508008C800198410703D54FF40061E16000E0E66012
S31508008C90800701D5A6601BE04FF48040A06017E06E
S31508008CA0E0680021C0F3CF02A068C0F34F0002437A
S31508008CB0204600F06FF938B101212046FFF75EFD26
S31508008CC084F84450012016E740F6FF70FFF740FE8F
S31508008CD041462046FFF752FD84F8445000200AE733
S31508008CE0443802400438014000D3CEFEC0E1E40017
S31508008CF040F1E9FD40787D0100796CFC005A62027A
S31508008D00001F0AFA80F0FA02F0B587B00068254914
S31508008D10884245D12448016841F000710160016824
S31508008D2001F000710191016841F0806101600168FC
S31508008D3001F080610191016841F0006101600068FD
S31508008D4000F000600190322002900224039400256E
S31508008D500495032605960B270697144802A900F0E2
S31508008D6057F986200290039404950596069702A95A
S31508008D700F4800F04DF920030290039404950596D8
S31508008D80069702A90B4800F043F94FF420500290C9
S31508008D90039404950596069702A9074800F038F942
S31508008DA007B0F0BD0080024030380240000802409B
S31508008DB00000024000040240001802402DE9F04776
S31508008DC00446914694F8440082281DD0822084F8EF
S31508008DD044002068026902F01C03228A4FF6FF75D8
S31508008DE005EAC2221A434FF4F86303EA81111143D4
S31508008DF021F0020141F00105056100F001FA06467D
S31508008E0001274FF480380FE00220BDE8F08700F014
S31508008E10F7F9801B404505D304F8447F00206070AD
S31508008E200320F2E720680569E807F0D12068406961
S31508008E3080B2C9F8000084F844700020E5E770B5F0
S31508008E40044694F84500012819D0012584F84550B0
S31508008E50022084F844002046FFF769FD2046FFF704
S31508008E6055FD2046FFF75CFC2046FFF751FC2046DF
S31508008E70FFF746FC04F8445F0020607070BD0220CE
S31508008E8070BDF0B5002390F84520012A11D00127BE
S31508008E9080F84570022280F84420002659B1C46A39
S31508008EA02268002A0CDA122100F8441F46700120B5
S31508008EB0F0BD0220F0BD00F8447F46700120F0BDE9
S31508008EC040F2F455A9420AD9B1FBF5F2B1FBF5FC1B
S31508008ED005FB1C1CBCF1000F02D0521C00E001224D
S31508008EE0012A44D1226842F040522260C26AC1F384
S31508008EF00C015160C16A0A6842F000420A60C16A00
S31508008F00C968C16235E0C46AD4F800C02CF0405C78
S31508008F10C4F800C033B9C46AD4F800C04CF0805C09
S31508008F20C4F800C0C46A6560541EA34214D1C46A5A
S31508008F30D4F800C04CF0005CC4F800C0C2F10104CB
S31508008F40C4EBC41404EB440401EB8404D0F82CC02D
S31508008F50C4F30C04CCF80440C46AD4F800C04CF03E
S31508008F60004CC4F800C0C46AE468C4625B1C93423F
S31508008F70C9D3016801F580514A69520705D504220B
S31508008F804A61016801F580514E6000F8447F4670D9
S31508008F900020F0BD2DE9F041044694F8440042282B
S31508008FA020D0422084F844002068036903F01C039B
S31508008FB0258A4FF6FF7606EAC5251D434FF4F86362
S31508008FC003EA8111294341F0020141F0010591B2FA
S31508008FD041612068056100F013F9064601274FF440
S31508008FE080380FE00220BDE8F08100F009F9801B07
S31508008FF0404505D304F8447F002060700320F2E75B
S3150800900020680569E807F0D184F84470EBE70000AA
S315080090102DE9F84F0022DFF8A491DFF8A0814FF080
S31508009020010E09F108094FF00F0C09F1040A0EFAAE
S3150800903002F60B683340B34271D14C68022C01D05A
S31508009040122C11D1D40800EB84073D6A5407E40EAC
S315080090500CFA04FB25EA0B05D1F810B00BFA04FB51
S315080090604BEA050BC7F820B0076854000325A5404E
S31508009070AF4391F804B00BF0030B0BFA04FB4BEA71
S31508009080070BC0F800B04F68012F05D0022F03D098
S31508009090112F01D0122F11D18768AF43D1F80CB028
S315080090A00BFA04FB4BEA070BC0F808B04768B7434E
S315080090B00E79C6F3001696403E434660C668AE4330
S315080090C08D68A5403543C5604C68E4006FD53C4CB7
S315080090D0256845F480452560246804F48044009496
S315080090E0384C22F003052544D5F808789407260F4E
S315080090F00CFA06F4A743344CA04201D100242EE012
S31508009100324CA04201D1012429E0314CA04201D1C0
S31508009110022424E02F4CA04202D103241FE046E09B
S315080091202D4CA04201D1042419E02C4CA04201D1B7
S31508009130052414E02A4CA04201D106240FE0294C4C
S31508009140A04201D107240AE0274CA04201D10824F5
S3150800915005E0264CA04201D1092400E00A24B440C7
S315080091603C43C5F80848D8F800409C434D68ED03D1
S3150800917000D51C43C8F80040104D2D1D2C689C4393
S315080091804E68B60300D51C432C60D9F800409C43B2
S315080091904D68ED0200D51C43C9F80040DAF80040D6
S315080091A09C434D68AD0200D51C43CAF80040521CCA
S315080091B0102AFFF43CAFBDE8F88F0000003C0140E0
S315080091C044380240003001400000024000040240DA
S315080091D000080240000C0240001002400014024041
S315080091E000180240001C02400020024000240240F1
S315080091F0002A01D081617047090481617047000027
S3150800920001488068704700004000002002488168D5
S3150800921002781144816070474000002010B5032091
S3150800922000F0DAF8002000F005F800F025F8002034
S3150800923010BD000070B504460D4D4FF47A712878BC
S31508009240B1FBF0F00B490968B1FBF0F000F00DFC3A
S3150800925008B1012070BD102C07D200222146501EED
S3150800926000F09AF86C60002070BD012070BD000007
S31508009270400000205400002010B586B04349086815
S3150800928040F080500860086800F080500090081D83
S31508009290026842F480420260006800F48040009050
S315080092A03A481038026842F001020260026802F089
S315080092B001020092026842F002020260026802F0AD
S315080092C002020092026842F004020260026802F09A
S315080092D004020092026842F008020260026802F084
S315080092E008020092026842F040020260006800F03C
S315080092F040000090086840F480200860086800F480
S3150800930080200090032000F067F800226FF00B0021
S31508009310114600F041F800226FF00A00114600F0ED
S315080093203BF800226FF00900114600F035F80022DC
S31508009330501F114600F030F80022101F114600F0A9
S315080093402BF80022901E114600F026F80022501E27
S31508009350114600F021F88020019001200290002497
S315080093600394049401A90A48FFF752FE4FF440708B
S315080093700190022002900394032004900720059090
S3150800938001A90448FFF744FE06B010BD4038024064
S3150800939000040240000C0240F0B40D460D4B1B6859
S315080093A0C3F30223C3F10704042C00D90424191DAE
S315080093B0072901D2002300E0DB1E012606FA04F184
S315080093C0491E294099409E40761E16403143F0BCFE
S315080093D000F04CBC0CED00E000F00701054A1068EF
S315080093E04FF6FF03184040EA01200349084310607E
S315080093F0704700000CED00E00000FA05F8B51948C2
S31508009400016841F080510160006800F080500090CA
S31508009410154C206840F480302060FFF7F1FE0546C1
S315080094204FF47A7606E0FFF7EBFE401BB04201D90F
S315080094300320F8BD6068C003F5D5206840F4003005
S315080094402060FFF7DDFE054606E0FFF7D9FE401B64
S31508009450B04201D90320F8BD60688003F5D5002025
S31508009460F8BD000040380240007000402DE9F04782
S3150800947004460D46002C17D0DFF83081D8F80000D6
S3150800948000F00F00A84211D2D8F8000020F00F0013
S315080094902843C8F80000D8F8000000F00F00A842DA
S315080094A004D00120BDE8F0870120FBE72068404E84
S315080094B0810712D5400703D5306840F4E050306084
S315080094C02078000703D5306840F460403060306883
S315080094D0A16820F0F000084330602078C0072ED03D
S315080094E0334960680839012806D0022809D0096876
S315080094F089070BD40120D5E70968890306D401201A
S31508009500D0E70968890101D40120CBE7316821F049
S31508009510030101433160FFF773FE074641F28839BC
S3150800952006E0FFF76DFEC01B484501D90320B9E7E1
S315080095303068616800F00C00B0EB810FF1D1D8F803
S31508009540000000F00F00A8420ED9D8F8000020F05D
S315080095500F002843C8F80000D8F8000000F00F00F4
S31508009560A84201D001209DE72078400705D530683C
S31508009570E16820F4E050084330602078000706D5FB
S315080095803068216920F4604040EAC100306000F08C
S315080095903BF83168074AC1F30311515CC8400649D4
S315080095A008600020FFF746FE00207BE7003C0240EB
S315080095B008380240DEB90008540000200148006857
S315080095C0704700005400002000B5FFF7F7FF044974
S315080095D00968044AC1F38221515CC84000BD0000F5
S315080095E008380240EEB9000800B5FFF7E7FF04495E
S315080095F00968044AC1F34231515CC84000BD000005
S3150800960008380240EEB9000810B51748006810F08F
S315080096100C01164816D04310042912D0082911D176
S31508009620114C241F216801F03F02216849020AD51E
S315080096302068C0F38810A0FB03010023FEF752FE42
S3150800964009E0184610BD21680023C1F38811A1FB63
S315080096500001FEF747FE2168C1F30141491C490094
S31508009660B0FBF1F010BD0000083802400024F400F9
S315080096702DE9F84F04464FF00008002C15D0207845
S31508009680DFF8C093A9F10407C007A7F1040560D065
S31508009690D9F80000C0F3810001280CD0D9F80000E1
S315080096A0C0F38100022803D00CE00120BDE8F88F42
S315080096B03868400206D5286880034AD5606870BBBA
S315080096C00120F3E76068B0F5803F11D0A8B1B0F586
S315080096D0A02F1BD0286820F480302860286820F442
S315080096E080202860606830B3FFF78AFD06461EE0D2
S315080096F0286840F480302860F4E7286820F4803031
S315080097002860286820F480202860EBE7286840F461
S3150800971080202860286840F480302860E2E718E056
S31508009720FFF76EFD801B642801D90320BEE7286871
S315080097308003F5D50DE0FFF763FD064606E0FFF763
S315080097405FFD801B642801D90320AFE728688003E2
S31508009750F5D4207880074BD5D9F8000010F00C0F07
S3150800976008D0D9F80000C0F38100022812D1386861
S3150800977040020FD42868800704D5E068012801D084
S31508009780012093E72868216920F0F80040EAC10023
S3150800979028602DE0E068C8B1286840F0010028601C
S315080097A0FFF72EFD064606E0FFF72AFD801B022876
S315080097B001D903207AE728688007F5D52868216942
S315080097C020F0F80040EAC100286011E0286820F07F
S315080097D001002860FFF714FD064606E0FFF710FDB6
S315080097E0801B022801D9032060E728688007F5D482
S315080097F02078000730D5DFF84CA260690AF16C0AB8
S31508009800A8B1DAF8000040F00100CAF80000FFF736
S31508009810F7FC064606E0FFF7F3FC801B022801D991
S31508009820032043E7DAF800008007F4D514E0DAF8F5
S31508009830000020F00100CAF80000FFF7E1FC064628
S3150800984006E0FFF7DDFC801B022801D903202DE77F
S31508009850DAF800008007F4D42078400775D5DFF8D9
S31508009860E4A10AF1380ADAF80000C0000CD4DAF8E4
S31508009870000040F08050CAF80000DAF8000000F056
S31508009880805000904FF00108DFF8BCB1DBF800000B
S31508009890C00514D4DBF8000040F48070CBF8000053
S315080098A0FFF7AEFC064606E0FFF7AAFC801B642815
S315080098B001D90320FAE6DBF80000C005F4D5DFF885
S315080098C084B1A0680BF1680B012814D0D0B1052823
S315080098D025D0DBF8000020F00100CBF80000DBF80B
S315080098E0000020F00400CBF80000A06870B3FFF772
S315080098F087FC06462BE0DBF8000040F00100CBF8B9
S315080099000000F2E7DBF8000020F00100CBF80000C9
S31508009910DBF8000020F00400CBF80000E5E7DBF8F0
S31508009920000040F00400CBF80000DBF8000040F02F
S315080099300100CBF80000D8E7FFF762FC811B41F273
S315080099408830814203D90320B0E61FE004E0DBF843
S3150800995000008007F0D510E0FFF752FC064608E045
S31508009960FFF74EFC811B41F28830814201D9032062
S315080099709CE6DBF800008007F2D4B8F1010F05D1A8
S31508009980DAF8000020F08050CAF80000A069E8B3B1
S31508009990D9F80010C1F38101022951D0022807D055
S315080099A0286820F080702860FFF72AFC044642E009
S315080099B0286820F080702860FFF722FC064606E03B
S315080099C0FFF71EFC801B022801D903206EE62868D3
S315080099D08001F5D454F81C0F4FF0FF336168E26834
S315080099E00843A16803EB5202890141EA0241084390
S315080099F0217C40EA0160217D40EA017038602868D0
S31508009A0040F080702860FFF7FBFB00E016E0044694
S31508009A1006E0FFF7F5FB001B022801D9032045E6FF
S31508009A2028688001F5D509E0FFF7EAFB001B022844
S31508009A3001D903203AE628688001F5D4002035E6E6
S31508009A40012033E6083802400070004004284FF031
S31508009A50E02104D0086920F004000861704708690D
S31508009A6040F0040008617047704710B5401EB0F119
S31508009A70807F01D3012010BD4FF0E02460610F21E3
S31508009A80601700F0F3F80020A0610720206100208D
S31508009A9010BD10B5FFF7E8FF10BD10B50446002C41
S31508009AA003D094F8690010B107E0012010BD00202A
S31508009AB084F86800204600F028F8242084F8690015
S31508009AC02068016821F001010160204600F026FBAC
S31508009AD0012818D0606A10B1204600F09CFA206868
S31508009AE0416821F4904141602068816821F02A018B
S31508009AF081602068016841F0010101602046BDE8E7
S31508009B00104000F0ECBA012010BD70472DE9F84F5F
S31508009B1004460D461646984694F86A00202802D050
S31508009B200220BDE8F88FFDB1F6B194F86800012867
S31508009B301CD001204C3420774FF00009C4F820903F
S31508009B402220A077FFF75CFB8246A681E681FF22EA
S31508009B5054F8440C4C3C4FF48057B8420DD1206958
S31508009B6030B1A4F85C201BE00120DAE70220D8E730
S31508009B7040F2FF10A4F85C0012E07F2118B1B0F1A2
S31508009B80805F08D00CE0206910B1A4F85C1007E0EB
S31508009B90A4F85C2004E0206928B13F20A4F85C0002
S31508009BA0B4F85C601CE0A4F85C10F9E7B4F85A0055
S31508009BB0401EA4F85A000022534620212046CDF81C
S31508009BC0008000F029FC08B10320AAE7A068B84283
S31508009BD001D1206978B12068406A304005F8010B48
S31508009BE0B4F85A000028E1D1202084F86A0084F8E5
S31508009BF06890002095E72068406A304025F8020BF7
S31508009C00EEE710B5FFF70AFB00F086F900F0F0F969
S31508009C10BDE81040AFF30080002202488021FFF71C
S31508009C20E7BA00000004024070B500F0DFF9044608
S31508009C300C4D6868201AB0F5FA7F0AD328780A4BC3
S31508009C4040B100202870002218468021FFF7D0FA7C
S31508009C506C6070BD01202870012218468021FFF72C
S31508009C60C7FAF5E760000020000402400907090E5C
S31508009C70002806DA00F00F0000F1E02080F8141D35
S31508009C80704700F1E02080F80014704710B50B48C3
S31508009C900078410611D480070FD509480068001DD1
S31508009CA00178FF2909D14078002806D1012100F062
S31508009CB00FF9BDE81040FEF7BDBC10BD7C000020C2
S31508009CC09000002010B500F0DFFD00F08FF9144C6D
S31508009CD000F5FA70206000F089F942F21071084424
S31508009CE0606001F0E9F800200E49088048800E49B6
S31508009CF0088048800D49088048804EF6030001F028
S31508009D001BF900F0FBFD04F1080000F0ADFD06218B
S31508009D1004F1080000F062FCBDE8104000F078BCD1
S31508009D20680000208C000020AC000020A80000205D
S31508009D302DE9F04700F0F6FD354D002708B32880D9
S31508009D404FF4006000F078FD324CA18988420AD1B0
S31508009D50012001F007F9288898B100F079FF00F092
S31508009D6005FE2F800DE040F6060000F065FDA1898E
S31508009D70884206D100F016FF288810B100F0F6FDDB
S31508009D802F8000F033F9244E3168884230D301F52C
S31508009D90FA7131600024DFF88480DFF88490C4EB20
S31508009DA0041008EB4000C9F80000022001F0DAF8B8
S31508009DB0288820B100F04CFF00F0D8FD2F80641CE5
S31508009DC0002CECD00024DFF85C80DFF85C9008EB10
S31508009DD08410C9F80000052001F0C4F8288820B1CD
S31508009DE000F036FF00F0C2FD2F80641C002CEED078
S31508009DF000F0FCF87168884207D342F210700844F4
S31508009E007060BDE8F04700F0D1BFBDE8F0870000FC
S31508009E10800000208832002068000020CA38002010
S31508009E2098000020E83800209C0000200B4A1068A3
S31508009E30C1B2C0F307231944C0F30743194401EB21
S31508009E401061002013181B79194489B2401C382860
S31508009E50F8D3C843401C80B27047000000000020B9
S31508009E6010B500F015F800280DD108490648086015
S31508009E70002000220B181A71401C3828FAD3BDE8B6
S31508009E80104000F039B810BDA2E742CE000000200D
S31508009E9010B50024054806490068884203D100F039
S31508009EA009F800B10124204610BD0000000000207A
S31508009EB0A2E742CE10B50024FFF7B8FF0349898F01
S31508009EC0884200D10124204610BD00000000002071
S31508009ED070B504460E460025FFF7DAFF38B1382C70
S31508009EE005D204482044067100F006F801252846E4
S31508009EF070BD00000000002010B5FFF797FF01496C
S31508009F00888710BD0000002010B5FFF77FF9BDE86F
S31508009F101040FFF7BEBD000010B594B01E4801689A
S31508009F2041F080510160006800F0805001901B48A4
S31508009F30016841F440410160006800F44040019026
S31508009F40012007900004089002240D9480010E90C9
S31508009F5008200F904FF4D87010901194129407A807
S31508009F60FFF786FB00B1FEE7FFF748FA00B1FEE708
S31508009F700F2002900394002004904FF4A0500590FF
S31508009F804FF480500690072102A8FFF76FFA0028C1
S31508009F9000D0FEE714B010BD403802400070004003
S31508009FA00E48016841F4700101600D48016841F0EE
S31508009FB0010101600A4A0021083211600268094B52
S31508009FC01A400260031D084A1A60026822F48022B9
S31508009FD0026003480C3001607047000088ED00E01D
S31508009FE000380240FFFFF6FE10300024FFF708B9DC
S31508009FF010B5FFF7E3FA4FF47A71B0FBF1F0FFF70B
S3150800A00034FD0420FFF722FD0022BDE81040501E53
S3150800A0101146FFF7C1B990F82410C90706D00168A0
S3150800A0204A68836A22F400321A434A6090F8241078
S3150800A030890706D501684A68C36A22F480321A433A
S3150800A0404A6090F82410490706D501684A68036BE8
S3150800A05022F480221A434A6090F82410090706D58C
S3150800A06001684A68436B22F400421A434A6090F832
S3150800A0702410C90606D501688A68836B22F48052C3
S3150800A0801A438A6090F82410890606D501688A68FA
S3150800A090C36B22F400521A438A6090F824104906CA
S3150800A0A011D501684A68036C22F480121A434A6083
S3150800A0B0016CB1F5801F06D101684A68436C22F429
S3150800A0C0C0021A434A6090F82410090606D50168AA
S3150800A0D04A68806C22F4002202434A60704738B509
S3150800A0E004460025E566FFF78BF8034620680068F6
S3150800A0F000070BD56FF07E400090002220464FF4F3
S3150800A100001100F089F908B1032038BD2020683411
S3150800A1106070A0702570002038BD00002DE9F04160
S3150800A1200446102100220025A3682069E669034336
S3150800A13060693043034320680668AB4F3E401E43C0
S3150800A140066020684368E66823F440533343436057
S3150800A150A369206A03432068866826F430661E438E
S3150800A1608660A24FCE022068A14BB84212D11B6866
S3150800A17013F0030306D0012B08D0022B04D0032BBF
S3150800A18001D105E00121A9E00221A7E00421A5E00B
S3150800A1900821A3E0974FB84212D11B6813F00C03AD
S3150800A1A006D0042B08D0082B04D00C2B01D105E0CF
S3150800A1B0002193E0022191E004218FE008218DE03F
S3150800A1C08D4FB84212D11B6813F0300306D0102BFE
S3150800A1D008D0202B04D0302B01D105E000217DE0EA
S3150800A1E002217BE0042179E0082177E0834FB84219
S3150800A1F012D11B6813F0C00306D0402B08D0802B61
S3150800A20004D0C02B6AD105E0002167E0022165E091
S3150800A210042163E0082161E0794FB84215D11B6833
S3150800A22013F4407309D0B3F5807F0AD0B3F5007FE5
S3150800A23005D0B3F5407F51D105E000214EE002215B
S3150800A2404CE004214AE0082148E06E4FB84215D197
S3150800A2501B6813F4406309D0B3F5806F0AD0B3F5D1
S3150800A260006F05D0B3F5406F38D105E0012135E020
S3150800A270022133E0042131E008212FE0624FB84281
S3150800A28015D11B6813F4405309D0B3F5805F0AD083
S3150800A290B3F5005F05D0B3F5405F1FD105E0002197
S3150800A2A01CE002211AE0042118E0082116E0574FA5
S3150800A2B0B84213D11B6813F4404308D0B3F5804F56
S3150800A2C009D0B34205D0B3F5404F07D105E00021C8
S3150800A2D004E0022102E0042100E00821E369B34218
S3150800A2E040D1092935D2DFE801F0050F19342134A8
S3150800A2F034342B00FFF768F94100606801EB500120
S3150800A300B1FBF0F082B225E0FFF76EF94100606814
S3150800A31001EB5001B1FBF0F082B21BE060683C49EA
S3150800A32001EB5001B1FBF0F082B213E0FFF76CF9D4
S3150800A3304100606801EB5001B1FBF0F082B209E020
S3150800A34060684FF4803101EB5001B1FBF0F082B246
S3150800A35000E0012522F00F00C2F3420108432168FC
S3150800A360C8603EE009293BD2DFE801F005111D3A35
S3150800A370263A3A3A3200FFF727F90146606801EBB8
S3150800A3805001B1FBF0F0216880B2C86029E0FFF700
S3150800A3902BF90146606801EB5001B1FBF0F021682A
S3150800A3A080B2C8601DE061681A4A02EB5102B2FB2E
S3150800A3B0F1F189B2C16014E0FFF726F90146606839
S3150800A3C001EB5001B1FBF0F0216880B2C86008E0EB
S3150800A3D0616806EB5102B2FBF1F189B2C16000E097
S3150800A3E001252846BDE8F081F369FFEF001001401A
S3150800A3F0903802400044004000480040004C0040AD
S3150800A400005000400014014000780040007C0040E5
S3150800A4100048E8010024F4002DE9F04104460E4600
S3150800A42017469846069D1DE0681C1BD02DB1FEF701
S3150800A430E7FEA0EB0800A84214D32068016821F4BF
S3150800A440D07101602068816821F0010181602020B7
S3150800A45084F8690084F86A00002084F868000320FC
S3150800A460BDE8F0812068C06936EA000004D0002003
S3150800A470B842D9D00020F3E70120F9E710B5002348
S3150800A480014604480122FFF741FB08B1002010BD30
S3150800A490012010BDE4310020FF2100F8011B7047A0
S3150800A4A035220270012242708170C01C704700007C
S3150800A4B032210170042141700249496AC0F802102C
S3150800A4C0801D7047543200203721017003214170E6
S3150800A4D001228270C17006210171401D704700007B
S3150800A4E036210170042141700249C969C0F8021079
S3150800A4F0801D70475432002010B58B185B1E0BE088
S3150800A5000C784A7802EB042292B2104480B2904248
S3150800A51001D2401C80B2891C9942F1D3994207D1D5
S3150800A52009780902084480B2884201D2401C80B2E8
S3150800A53010BDFFF75BBD00002DE9F0410446012080
S3150800A54020706070164D287EA0700020E070154EB1
S3150800A5503168616020818021618113490968E16061
S3150800A56020616061A06104F11C00D5E90512074667
S3150800A570FDF75BFFA869C0F110013844FDF7A2FF9B
S3150800A580402104F12C00FDF79DFF802104F16C00A9
S3150800A590FDF798FF7068C4F8EC00BDE8F08100008C
S3150800A5A054320020F6B900088C00002000F03AB8B2
S3150800A5B00749828C0A80C28C4A800649028D0A8025
S3150800A5C0428D4A800449028E0A80408E4880704730
S3150800A5D08C000020AC000020A800002038B50B4CE9
S3150800A5E06061A1610025A5704FF6FF70ADF8000007
S3150800A5F0ADF802004FF48641684601F07FF96060C5
S3150800A60010B14FF488418180258038BD543200202E
S3150800A6100021024801804180704700008C0000201C
S3150800A620704700002DE9F84F0120814C814D002626
S3150800A6304FF493784FF002094FF47A774FF0030AF4
S3150800A640218804F1080242F2107B009241454FD05E
S3150800A65009DCB1B1A1F580710F391FD0012921D0CC
S3150800A66016290AD141E0A1F5807155397DD0012915
S3150800A6707CD015297BD016297AD026800220BDE801
S3150800A680F88F0120A070276100F004FA216900986C
S3150800A69000F03FFA002040F20F112180F0B34FF48A
S3150800A6A0887020802878800703D4009800F024FA60
S3150800A6B0A8B32878800703D500F08CF9022836D08D
S3150800A6C020694EF66021884201DA40002061A078B0
S3150800A6D00228D9D1276100F0F5F92169009800F020
S3150800A6E018FA002040F22511218018B3A4F800803A
S3150800A6F02878800703D4009800F0FEF9E0B128789E
S3150800A700800703D500F066F9052817D02069584553
S3150800A71037DC00F57A702061A07801E003E004E0F8
S3150800A7200328D8D10CE00320A9E70020A7E784F87E
S3150800A7300290CFE70320A2E70020A0E784F802A052
S3150800A7403B48FFF735FF208C00F076F84FEA0048C3
S3150800A750608C00F071F840EA080040084FF00042AB
S3150800A76000EB4001C1EBC01103E018E01BE02FE04D
S3150800A77032E0B2EBC10F07D94FF47A714843206132
S3150800A78005E0268000207AE76FF000402061216905
S3150800A790009800F0BEF9002040F25511218098B3C8
S3150800A7A04FF4AB702080009800F0A6F968B384F8DF
S3150800A7B002902761FFF72CFFFFF732FF00F082F9BE
S3150800A7C02169009800F0A5F900204FF4B5712180A1
S3150800A7D000B340F26B1020802878800703D40098D5
S3150800A7E000F08AF9C0B12878800703D500F0F2F89E
S3150800A7F0052813D02069584516DC00F57A702061C3
S3150800A800A0780328DAD10BE000E001E0032036E760
S3150800A810002034E7032032E7002030E784F802A05E
S3150800A8200348FFF7C5FE8EE72680002027E70000CD
S3150800A830543200207C000020010241EA102080B238
S3150800A8407047FFF7DEF9FFF70BFBFFF73BFAFDF75B
S3150800A85005FF00210846FFF73BFBFFF7E5F9FFF781
S3150800A86067FAFDF7F9FEF8E706490A7802704A78AA
S3150800A87042708A788270CA78C2700A7902714979F8
S3150800A880417170474C00002010B517480821017027
S3150800A89000224270272181706921C1705B210171F4
S3150800A8A0452141711249114B0B6001234B600A8205
S3150800A8B048618A61CA61D80508620846FEF70EF93A
S3150800A8C00B4904230B4A0A48C831FEF78AF80A4A94
S3150800A8D004230748A2F58071FEF74CF8BDE810403E
S3150800A8E00348FEF7ACBA00004C0000200080024086
S3150800A8F0B8000020D01900200002002007480849A7
S3150800A90002780A7042784A7082788A70C278CA7069
S3150800A91002790A7140794871704700004C0000209E
S3150800A9207600002070B500250E48FEF797F8B8B9EE
S3150800A9300C4CA08F85B2216C0B482A46FDF775FD95
S3150800A940216B086840F0004008600020A063216879
S3150800A95001F580514A69120602D580224A6188604B
S3150800A960284670BDB8000020883200202DE9F04145
S3150800A9700126154FFD6AFFF739FB00F1FA0405E0D9
S3150800A980FFF734FBA04201D9002602E02868002818
S3150800A990F6DB012E0BD10D480488F86A806822463A
S3150800A9A00B49FDF742FD08482146FEF76AFA386862
S3150800A9B000F580504169890603D5202141610021AF
S3150800A9C04160BDE8F0810000B8000020800000204A
S3150800A9D08832002070B50F480468207802280DD107
S3150800A9E00D490422201DFDF7F4FC38B90B4D04F17E
S3150800A9F01C00D5E90512FDF7ECFC08B1002070BD76
S3150800AA00206968620648018804F1F000BDE87040D4
S3150800AA1000F008B890000020F6B90008543200206B
S3150800AA208000002010B544180023194A29E001784F
S3150800AA30332920D006DC01290BD003290DD006299D
S3150800AA401CD10EE0352910D0362910D0FF2915D192
S3150800AA501BE0D0F80210916210E0D0F802101163E2
S3150800AA600CE0D0F80210D16208E0837806E0D0F84E
S3150800AA700210D16102E0D0F8021011624178801C00
S3150800AA800844A042D3D3184610BD184610BD00008E
S3150800AA905432002070B50A4D2C682046FFF74CFD4D
S3150800AAA0012104F1F000FFF7FBFCFFF70DFDFFF7AE
S3150800AAB0F3FC01462868BDE87040091A00F00ABF91
S3150800AAC09000002070B50B4D2C682046FFF734FD2A
S3150800AAD0032104F1F000FFF7E3FCFFF701FDFFF7A0
S3150800AAE0E7FCFFF7D9FC01462868BDE87040091A5B
S3150800AAF000F0F0BE9000002010B50446FFF719FDDF
S3150800AB002168401A6168884201DB012010BD0020D7
S3150800AB1010BD10B504466160FFF70BFD206010BD3F
S3150800AB2030B5144DC2780A44D4B2EC70827802EB80
S3150800AB301122D2B2AA7043786B7000782870B2EBF3
S3150800AB40112F05D25B1CDBB26B700BB9401C287049
S3150800AB50C8B284420DD2521CD0B2A870002808D1BF
S3150800AB606878401CC0B26870002802D12878401C5A
S3150800AB70287030BDA400002010B5094C0146E069D4
S3150800AB800830FFF7CDFFE06904F128010A78027260
S3150800AB904A7842728A788272C978C17210BD0000FA
S3150800ABA07C0000202DE9F047254D002029882A2918
S3150800ABB002D22880BDE8F08728804FF40076214C21
S3150800ABC0214F224602F11601B4F81490881DB2F8F6
S3150800ABD026C0B7F80080B9F5807F128D7B8809D02A
S3150800ABE0B145E7D1C445E5D19A42E3D1BDE8F0477E
S3150800ABF000F0FEB8C445DDD19A42DBD100F0F8F882
S3150800AC00A682D4F816002062618BA1840F4B1A68BD
S3150800AC10C4F816209B886383C4F8062063812060E5
S3150800AC20A180A08BE084E08B20853888A083788873
S3150800AC30E0834FF4C160A0812A202880BAE700008B
S3150800AC4080000020883200208C000020760000203A
S3150800AC502DE9F05FDFF82CA14FF6FF724A4B5046FC
S3150800AC60BAF81E10008C9C8891421D6809D1904242
S3150800AC7007D146480168CAF800108088AAF8040077
S3150800AC803FE0434B434F1A88B7F80090B7F8028065
S3150800AC9001EA0206404F09EA0202964206D15A889C
S3150800ACA000EA020308EA0202934205D03B480188FB
S3150800ACB039804088788001E0398078804FF0000B31
S3150800ACC0354B1B1F83F800B03E88DFF8D4C07F8859
S3150800ACD0197801EB41000CEB80000288964202D1FC
S3150800ACE04288974204D0491CC9B219700829EFD383
S3150800ACF01978082912D04168CAF800100089AAF8FC
S3150800AD000400CAF80650AAF80A400820AAF80C0057
S3150800AD10244801880E310180BDE8F09F1948FF22BA
S3150800AD200621FDF7C7FBCAF820B0AAF824B0CAF86E
S3150800AD300650AAF80A40CAF81650AAF81A40AAF8FD
S3150800AD402660AAF82870AAF81C90AAF81E804FF464
S3150800AD508070AAF81400AAF80E000820AAF81000B5
S3150800AD6006208AF8120004208AF813004FF4C160FE
S3150800AD70AAF80C000C490348363008602A2109480D
S3150800AD800180C9E78832002076000020FEB9000855
S3150800AD90AC0000208C000020B4000020A800002091
S3150800ADA0283900208000002090000020F0B50E4AC7
S3150800ADB09078401CC5B29570002313700B4E11781D
S3150800ADC001EB410006EB8000048847883C4304D029
S3150800ADD0847A2C1B782C00DB0360491CC8B21070DF
S3150800ADE00828ECD3F0BD0000B00000202839002068
S3150800ADF02DE9F0412E4F4FF0000C87F800C02D4E7C
S3150800AE003B7803EB430206EB8202148884B155882B
S3150800AE1075B1B0F80080A0450AD14488AC4207D184
S3150800AE200868506088881081B8789072BDE8F0810B
S3150800AE305B1CDAB23A70082AE2D387F800C03B787E
S3150800AE4003EB430206EB820214880CB9548824B13A
S3150800AE505B1CDBB23B70082BF1D33B78082B1DD16A
S3150800AE6087F803C087F801C087F800C0BC783A782D
S3150800AE7002EB420306EB8303FD789B7AE31AAB42A7
S3150800AE8001DDFB707A70521CD2B23A70082AEED3F2
S3150800AE907A783A7002EB420206EB8202006810608A
S3150800AEA00868506088881081B8789072BEE70000FC
S3150800AEB0B00000202839002010B5154A002151702D
S3150800AEC002F10803507823F81010401CC0B25070E5
S3150800AED00028F7D051700F4B5078C0EB001403EBE5
S3150800AEE044046176401CC0B250700028F4D04FF478
S3150800AEF0806090815170074B1E33507803EB8014A5
S3150800AF00A180401CC0B250700028F6D010BD0000C9
S3150800AF107C000020CA38002010B5064914220020FB
S3150800AF20FFF7EAFA18B1BDE81040FFF785BC4FF6FF
S3150800AF30FF7010BD9632002010B5094A00215170E5
S3150800AF4002F10803517833F811402CB1491CC9B2F3
S3150800AF5051700029F6D010BD517823F8110010BDA4
S3150800AF607C0000202DE9F05FF84FFC690026F84DBB
S3150800AF70042805F1360A77D0C7F814A0C7F818A030
S3150800AF8003284FF0010B4FF0100909D0022814D0FE
S3150800AF90052805F12A047BD0A87B452843D185E0FE
S3150800AFA0607E00F00F000328F8D1208A0028F5D12A
S3150800AFB008203870FEF76AFEA6E3E4492431C8780B
S3150800AFC0401C10F0FF00C8700ED18878401C10F0A5
S3150800AFD0FF00887008D14878401C10F0FF004870C0
S3150800AFE002D10878401C0870BE80FE80607E072863
S3150800AFF012D0052810D0002815D0218AA9B3A07E22
S3150800B000411EA1760FD2E07E082824D0617E02294F
S3150800B0100AD0012908D009E0A07E401CC0B2A0765B
S3150800B0207828BBD16676ECE0052814D0042800D928
S3150800B030042003218140A176E07E401CE076607EF4
S3150800B04000F00F000928EED2DFE800F0DBFC11144F
S3150800B050FBDBFBDBFB00667680203870FEF716FE0E
S3150800B060142085F82F00D2E39EE008E010E085F86A
S3150800B0702F60E4E104203870FEF708FE62E300F072
S3150800B0800F000328CFD108203870FEF7FFFD3BE3F9
S3150800B090386A80880028C6D0FE617C61BC61FE8063
S3150800B0A0BE8008203870FFF781FA7DE0297C687C2D
S3150800B0B000EB0120B9888842B5D8B880287D80067B
S3150800B0C0B1D1687D0028AED1A048103001884088EB
S3150800B0D001B928B1EA8B8A42A5D1298C8142A2D12D
S3150800B0E0FFF71AFF4FF6FF7840459CD1E87D062802
S3150800B0F004D011280FD0012895D115E000F0FAFBED
S3150800B100404590D1934CA8466A8C6B8B2146B5F87E
S3150800B1101CC0A88C9BE0B8881C38B8808D481E30A7
S3150800B120386200F1400269E095F822000828A9D1A2
S3150800B13085F822604FF6F771A88C884202D3093049
S3150800B140A88401E00830A884688BE883A88B288443
S3150800B1507E481030018869834088A883B5E38188D2
S3150800B160F1B3AB8C8B4247D1C18829B16B8C8B422A
S3150800B17002D0B1F58A4F3FD1018809B943885BB13E
S3150800B180414502D14388434506D06B8B8B4233D168
S3150800B190A98B438899422FD1FE61022038707C61C1
S3150800B1A0BC61FE80FFF702FAF988002929D001F16F
S3150800B1B01C00B880020A2A746874386A027AAA756A
S3150800B1C01122EA750831C1F3072242EA0121E9840E
S3150800B1D02E8581886984C188A9845C49103100E07C
S3150800B1E00AE00A886A834988A9830188E98340882E
S3150800B1F02884C7F814A058E340303862386A904269
S3150800B200ADD33AE394F819A0BAF1000F1ED0B4F8FA
S3150800B21004A050451AD1B4F806A0524516D1B4F880
S3150800B22000A0534512D1B4F802A0D4450ED1FC6152
S3150800B2303E7098F82F0041077CD566762020387036
S3150800B24001E02DE2F9E0FEF721FD16E31E348C42FB
S3150800B250D8D998F82F2002F03F02022A10D1F88197
S3150800B2607E703A4B08337A7833F81240844202D11A
S3150800B27000247E705FE0521CD2B27A70002AF2D0A7
S3150800B28098F82F004007BCD4142088F82F002820EF
S3150800B290B880502088F82E0098F8293098F82D00A4
S3150800B2A088F8290098F8281098F82C0088F82800BB
S3150800B2B088F82C1098F8272098F82B0088F827008B
S3150800B2C088F82B2098F82600787098F82A4088F88D
S3150800B2D0264088F82A005B1C13F0FF0388F82D30F7
S3150800B2E00ED1491C11F0FF0188F82C1008D1521C08
S3150800B2F012F0FF0188F82B1002D1401C88F82A00AA
S3150800B300B8F82200F881B8F82410A8F82210A8F88E
S3150800B3102400B8F81A00A8F81E00B8F81C00A8F807
S3150800B32020000A4810300188A8F81A104088A8F8A2
S3150800B3301C00ABE2AAE07A78C2EB021001EB4000EF
S3150800B340437E4BB1072B0DD013E000007C00002094
S3150800B35088320020CA3800207878C0EB001001EB4C
S3150800B36040040BE024B1837E94F81AC0634500D9E3
S3150800B3700446521CD0B278700028DCD0002C71D05C
S3150800B380BA46FC610320A0762076A6750420E075EF
S3150800B390E676B8F82400A080B8F82200E080B8F86D
S3150800B3A01A002080B8F81C00608084F819B0F948A3
S3150800B3B001782173417861738178A173C078E0734D
S3150800B3C0A4F810B098F82900E07298F82800A0723E
S3150800B3D098F82700607298F8260020720120FFF777
S3150800B3E0CBFB98F82E0000F0F001502925D98AF8F1
S3150800B3F001606FF0040101EB101319E008EB00027D
S3150800B40092F836108AF80210B9B1012902D0022939
S3150800B41004D007E0401C8AF8010009E092F83710CA
S3150800B420042920D092F8371039B108448AF8010067
S3150800B4309AF80100B0EB830FE0DB85F82F902E35E4
S3150800B440687840F00200687002202872042068724A
S3150800B4500620A8720A20E8722C20B880602005F819
S3150800B4602E09D9E1FEE09AF8010092F83810404416
S3150800B47090F8390040EA0120AAF80E0040F20A6165
S3150800B480884200D908466082A082D6E798F82E102E
S3150800B490090989007970BA88511A143989B2B980AC
S3150800B4A0627E02F00F02022A03D100F03F02122A3E
S3150800B4B017D009B9810714D098F826104346227A7E
S3150800B4C091427DD193F82710627A9142F9D193F887
S3150800B4D02810A27A9142F4D193F82910E27A91427F
S3150800B4E0EFD1C006C2463DD5218AD9B304F10C0076
S3150800B4F0FFF716FBA74B9AF82A101B1D18788142EE
S3150800B50030D19AF82B20D64659788A422AD19EF805
S3150800B5102CC09A78944525D19EF82DC0DB789C4599
S3150800B52020D120736173A273E373E07EA8B9207EED
S3150800B530A17E401AA17DA0EBD10040B20144C9B258
S3150800B540A175002801DA404240B2E27DA0EB9200E4
S3150800B5501044E07500EBD100207687F800B0207E15
S3150800B560A0762682607E00F00F0109297AD2DFE8EC
S3150800B57001F07905177AF8F7F627F5003878C00745
S3150800B58070D003206076402038702682B88818B1BB
S3150800B59042213970FFF7F0FAFE80FEF777FBB3E039
S3150800B5A03878C00705D09AF82F0000F03F00122817
S3150800B5B007D020203870FEF769FBF86946765FE603
S3150800B5C023E19AF82E0000F0F001502920D97E7068
S3150800B5D06FF0040101EB101316E00AEB000292F873
S3150800B5E03610B970A1B1012902D0022903D006E0AC
S3150800B5F0401C787008E092F83710042921D092F898
S3150800B600371029B1084478707878B0EB830FE4DBFB
S3150800B610032060769AF8260020729AF8270060724E
S3150800B6209AF82800A0729AF82900E0720120FFF71C
S3150800B630A3FA422038702682BE80FE80FEF726FBDB
S3150800B64062E0787892F83810504490F8390040EA69
S3150800B6500120F88140F20A61884200D908466082D2
S3150800B660A082D5E746E09AF82F10CA071CD0C20672
S3150800B6701AD4208AF0BBB888401C80B2FFF77CFA3F
S3150800B680387840F010003870B98811B140F00200DF
S3150800B6903870FEF7FBFAA4F810B008206076E67654
S3150800B6A0112085F82F00B2E089060BD59AF83420C8
S3150800B6B09AF8351041EA02217A690A447A61BA8809
S3150800B6C0511AB980B98841B1C00606D4387840F015
S3150800B6D0020038700846FFF74FFA9AF830109AF8C1
S3150800B6E0310000EB012080B2F881A18A814200D3A3
S3150800B6F010B900E04DE0F981F88960823878800752
S3150800B70047D0FE80FEF7C2FA3878810605D5FE8056
S3150800B7106676142085F82F0079E0C10609D5FE80E3
S3150800B720A4F810B004206076E676112085F82F007C
S3150800B7306DE0F98829B1C00700D02682208A88B131
S3150800B740F880E676B8697861F88890B1208A80B181
S3150800B7502830B880182085F82F005AE011E086E0D6
S3150800B7603EE019E0608A884200D2F880F888208294
S3150800B770E7E7387880070CD52820B88085F82F9019
S3150800B78047E03878C00778D0667687F80090FEF7E5
S3150800B7907DFA72E0A0000020B88808B1FFF7ECF93E
S3150800B7A09AF82F00C00711D03878C00704D00720B0
S3150800B7B06076A676268201E0062060760120FFF7ED
S3150800B7C0DBF987F80090FEF761FA1EE03878C007C3
S3150800B7D003D00520607626824FE0B888A8B94CE0E9
S3150800B7E0B88808B1FFF7C8F99AF82F00C0070AD039
S3150800B7F007206076A6760120FFF7BEF987F8009045
S3150800B800FEF744FA01E0B88880B388F82F9028201C
S3150800B810B880502085F82E001835207AA874607AEA
S3150800B820E874A07A2875E07A6875207BA873607B2F
S3150800B830E873A07B2874E07B6874062005F8010C81
S3150800B840A1886981E188A98121490A886A8049888D
S3150800B850A9802188E98061882981183D617EC90609
S3150800B8600FD585F8316085F830600FE005E0387847
S3150800B870C00702D007206076A676BE803E70BDE877
S3150800B880F09F85F830000A2085F831004020A87519
S3150800B890B888010A2974687485F8356085F83460B3
S3150800B8A06E8600F027F8C04368864520A873EE73B5
S3150800B8B06E752E757889401C7881010AA974E8741A
S3150800B8C02E83FFF729FBC04328833E70D7E7000085
S3150800B8D08C0000200346002908DD05488AB2C2808C
S3150800B8E08069834202D01946FCF79FBD7047000065
S3150800B8F07C000020062000F04DB800002DE9F0413C
S3150800B90004460F46214B0025214A4FF4FA484FF4C6
S3150800B91080569089401C80B29081404500D396811C
S3150800B92055709089FEF788FF0146507803EB801C16
S3150800B930BCF804C06145ECD0401CC0B25070002869
S3150800B940EFD000205570517803EB8116B688A6B162
S3150800B950491CC9B251700029F5D090B191890A02E3
S3150800B96042EA11218180C7806CB1218801806188F3
S3150800B970418040210172BDE8F081507803EB8010C8
S3150800B980EBE70020F7E70560F3E70000E83800205A
S3150800B9907C00002010B50E496FF013034A7C097C21
S3150800B9A003EB012111448CB2204480B208490822D5
S3150800B9B01A31FEF7A1FD064922462231FEF79CFD03
S3150800B9C018B1BDE81040FEF737BF4FF6FF7010BD3F
S3150800B9D0883200204FF04070E1EE100A70470000F0
S3150800B9E00000000000000102030406070809000021
S3150800B9F0000001020304ADDE122363825363FFFFD6
S3150800BA00FFFFFFFF24BA000840000020780000006E
S3150800BA10388200089CBA0008B8000020303F0000B1
S3150800BA205482000801000000100000000000000019
S3150800BA3000000000000000000024F40000000000E0
S3150800BA4000000000000000000000000000000000E8
S3150800BA5000000000000000000000000000000000D8
S3150800BA6000000000000000000000000000000000C8
S3150800BA7000000000000000000000000000000000B8
S3150800BA8000000000000000000000000000000000A8
S3110800BA900000000000000000000000009C
S705080081FD74
